:020000040800F2
:100000000080003011080008E1040008E104000845
:10001000E1040008E1040008E10400080000000019
:10002000000000000000000000000000E3040008E1
:10003000E304000800000000E30400088107000852
:10004000E1040008E1040008E1040008E1040008FC
:10005000E1040008E1040008E1040008E1040008EC
:10006000E1040008E1040008E1040008E1040008DC
:10007000E1040008E1040008E1040008E1040008CC
:10008000E1040008E1040008E1040008E1040008BC
:10009000E1040008E1040008E1040008E1040008AC
:1000A000E1040008E1040008E1040008E10400089C
:1000B000E1040008E1040008E1040008E10400088C
:1000C000E1040008E1040008E1040008E10400087C
:1000D000E1040008E1040008E1040008E10400086C
:1000E000E1040008E104000800000000E104000849
:1000F000E1040008E1040008E1040008E10400084C
:10010000E1040008E1040008E1040008E10400083B
:10011000E1040008E1040008E1040008E10400082B
:10012000E1040008E1040008E1040008E10400081B
:10013000E1040008E1040008E1040008E10400080B
:1001400000000000000000000000000000000000AF
:10015000E1040008E1040008E1040008E1040008EB
:10016000E1040008E1040008E1040008E1040008DB
:10017000E1040008E1040008E104000800000000B8
:10018000E1040008E1040008E1040008E1040008BB
:10019000E1040008E1040008E1040008E1040008AB
:1001A000E1040008E1040008E10400080000000088
:1001B000E1040008E1040008E1040008E10400088B
:1001C000E1040008E1040008000000000000000055
:1001D0000000000000000000E10400080000000032
:1001E000000000000000000000000000000000000F
:1001F0000000000000000000E1040008E104000825
:10020000E1040008E104000800000000E104000827
:10021000E1040008E1040008E1040008E10400082A
:10022000E104000800000000E104000800000000F4
:10023000E1040008E104000800000000E1040008F7
:10024000E1040008E1040008E1040008E1040008FA
:10025000E1040008E1040008E1040008E1040008EA
:10026000E1040008E1040008E1040008E1040008DA
:10027000E1040008E1040008E104000800000000B7
:10028000E1040008E1040008E1040008E1040008BA
:1002900000000000E1040008E10400080000000084
:1002A00000000000E1040008E1040008E104000887
:1002B000E1040008E1040008E1040008E10400088A
:0C02C000E1040008E1040008E10400086B
:1002CC0044F20041C5F602010869C0F3C2000328DC
:1002DC0014D002280DD090BB0868800649F20000AB
:1002EC00C0F2D03058BF70470968C1F3C101C84093
:1002FC00704747F64000C0F27D1070478A6A886AE2
:10030C00C0F3051CC86ABCF1000F4B6B04BF002086
:10031C00704700F0010002F003024042022A00EA9A
:10032C00D3006FF35F3000EE100AB8EE400A0BD02A
:10033C006AB9086880060DD49FED221A17E040F6C2
:10034C000010C0F23D0070479FED1D1A0FE09FEDAD
:10035C001B1A0CE0086849F20002C0F2D032C0F35C
:10036C00C10022FA00F001EE100AB8EE411A086B37
:10037C009FED153A6FF35F2002EE100A086BC0F385
:10038C004620B8EE422A013000EE032A00EE10CAD5
:10039C00B7EE003AB8EE400A81EE000A32EE031ACC
:1003AC0020EE010A01EE100AB8EE411A80EE010AA5
:1003BC00BCEEC00A10EE100A704700BF0024744A4D
:0C03CC0020BCBE4B0024744C0000003923
:1003D800034C206804348047FBE700F003F8FEE78D
:0403E80038080008C9
:1003EC0084B04EF6245401200090CEF20004BFF3EA
:1003FC005F8F206820F480302060002020670190FF
:10040C0048F21F70029040F201100390684600F011
:10041C009CF805202067206840F480302060BFF3F2
:0E042C004F8FBFF36F8F00F057F800F0B9F854
:10043A004EF6885042F20003CEF20000C5F20023C5
:10044A00026842F470020260186800F00F00062881
:10045A0004D81868072262F30300186044F20040C7
:10046A004EF67F51C5F60200CEF6F621026842F03A
:10047A000102026000220261D0F800C001EA0C0108
:10048A0001601968090705D519684FF0070C6CF364
:10049A000301196040F200218261C0F20221C261A7
:1004AA00026281620021C0F2FF11C16240F2802122
:1004BA00C0F20111016342638163C2630164426451
:1004CA00016821F480210160026603F5005043F2BD
:0604DA00D2010160704731
:0204E000FEE735
:0204E200704761
:1004E40010B582B04EF60C504FF6FF02CEF200006B
:1004F40044F21844C5F602040168114040F2003287
:10050400C0F2FA5211430160FFF7DEFE216840F6A3
:100514002802C0F60002C1F30321515C226801F0F5
:100524001F01C84040F20801C3F2000108600F2017
:1005340000F02CF958B9D4F8DC0040F00200C4F8FB
:10054400DC00D4F8DC0000F002000190019802B055
:0205540010BDD8
:1005560010B54EF698514378CEF2000190F800C0DF
:100566000B608B6823F001038B6043684B60037B51
:10057600C27A90F80AE0447B120642EA0372837B51
:1005860042EACE4EC27B4EEA844E447A4EEA434E4F
:10059600007A4EEA024E4EEA042E4EEA400040EA47
:0605A6000C00886010BD8E
:1005AC0010B582B044F60C01C5F6020108680A6861
:1005BC00400740F20000C3F200000DD5022363F3A4
:1005CC0002020A60026851F8083C9B0404D40368D8
:1005DC009B1AB3F57A7FF6D900220192CA680123DF
:1005EC0063F38F32CA60CA6802F440420192019AE6
:1005FC00CA689204FCD544F20044C5F60204216991
:10060C0011F03802A16A13D0182A08BF5FEA817171
:10061C000ED0216841F0010121F018012160016820
:10062C002268520714D40268521A032AF8D30EE037
:10063C002168216841F0010121F018012160016855
:10064C002268520704D40268521A022AF8D972B6E8
:10065C0042F2000C6268C5F2002C402363F31E6268
:10066C006260DCF8002012070CD1DCF800200123BA
:10067C0063F30302CCF80020DCF8002002F00F0238
:10068C00012A76D1A269E269E269226AA269A269A9
:10069C0022F47062A261226852076AD5226941F283
:1006AC00883322F0070222610268216911F0380FA9
:1006BC0004D00168891A9942F7D95AE0A069000759
:1006CC001EBFA06920F00F00A061DCF8000010F044
:1006DC000E0F0CD0DCF80000012161F30300CCF804
:1006EC000000DCF8000000F00F00012841D1A069E7
:1006FC0010F0700F1EBFA06920F07000A061E069BF
:10070C0010F0700F1EBFE06920F07000E061E0692E
:10071C0010F4E06F1EBFE06920F4E060E061206A35
:10072C0010F0700F1EBF206A20F070002062FFF7DF
:10073C00C7FDA16940F62802C0F60002C1F30321EF
:10074C00515C40F20402C3F20002A36940F20803B8
:10075C0001F01F011278C3F2000320FA01F11020FE
:10076C00002A196018BF0F2000F00CF808B902B06D
:04077C0010BD72B684
:1007800040F20000C3F200000168013101607047CF
:1007900040F2080144F6D352C3F20001C1F26202F2
:1007A0000968A1FB02124FF0FF3101EB9212110E0A
:1007B00001D0012070474EF210030F28CEF2000343
:1007C0004FF0010003F6FC4C5A604FF0F0028CF839
:1007D00017204FF0070299601A6088BF7047DCF855
:1007E0000020C943C2F3022282F00703042B28BF72
:1007F00004239940C943033A28BF914009018CF86A
:10080000171040F20401C3F2000108700020704785
:10081000FFF713FE4EF68850CEF20000016851F447
:0808200070010160FFF7D8FD33
:100828000000000000000000010203040607080998
:100838005D08000800000030050000006F0800088F
:10084800080000305808000804000000E30300080E
:040858000090D00339
:10085C00206861680834002200E042540139FCD55C
:02086C007047D3
:10086E0020686168A2680C3401E08B5C8354013A05
:04087E00FBD57047EF
:0400000508000811D6
:00000001FF
